BL51 BANKED LINKER/LOCATER V4.13                                                        12/03/2007  00:32:50  PAGE 1


BL51 BANKED LINKER/LOCATER V4.13, INVOKED BY:
C:\KEIL\C51\BIN\BL51.EXE main.obj TO Table_lamps RAMSIZE (256)


MEMORY MODEL: SMALL


INPUT MODULES INCLUDED:
  main.obj (MAIN)
  C:\KEIL\C51\LIB\C51S.LIB (?C_STARTUP)


LINK MAP OF MODULE:  Table_lamps (MAIN)


            TYPE    BASE      LENGTH    RELOCATION   SEGMENT NAME
            -----------------------------------------------------

            * * * * * * *   D A T A   M E M O R Y   * * * * * * *
            REG     0000H     0008H     ABSOLUTE     "REG BANK 0"
            DATA    0008H     0002H     UNIT         ?DT?MAIN
                    000AH     0016H                  *** GAP ***
            BIT     0020H.0   0000H.1   UNIT         ?BI?MAIN
                    0020H.1   0000H.7                *** GAP ***
            IDATA   0021H     0001H     UNIT         ?STACK

            * * * * * * *   C O D E   M E M O R Y   * * * * * * *
            CODE    0000H     0003H     ABSOLUTE     
            CODE    0003H     001DH     UNIT         ?PR?DEC?MAIN
            CODE    0020H     001BH     UNIT         ?PR?ADD?MAIN
            CODE    003BH     001AH     UNIT         ?PR?MAIN?MAIN
            CODE    0055H     0017H     UNIT         ?PR?DRIVE?MAIN
            CODE    006CH     0015H     UNIT         ?PR?_DELAY1MS?MAIN
            CODE    0081H     0013H     UNIT         ?PR?OPEN?MAIN
            CODE    0094H     0013H     UNIT         ?PR?CLOSE?MAIN
            CODE    00A7H     0011H     UNIT         ?PR?INIT?MAIN
            CODE    00B8H     0010H     UNIT         ?PR?_DELAY?MAIN
            CODE    00C8H     000CH     UNIT         ?C_C51STARTUP



OVERLAY MAP OF MODULE:   Table_lamps (MAIN)


SEGMENT
  +--> CALLED SEGMENT
---------------------
?C_C51STARTUP
  +--> ?PR?MAIN?MAIN

?PR?MAIN?MAIN
  +--> ?PR?INIT?MAIN
  +--> ?PR?OPEN?MAIN
  +--> ?PR?DRIVE?MAIN
  +--> ?PR?CLOSE?MAIN
  +--> ?PR?ADD?MAIN
  +--> ?PR?DEC?MAIN

BL51 BANKED LINKER/LOCATER V4.13                                                      12/03/2007  00:32:50  PAGE 2


?PR?OPEN?MAIN
  +--> ?PR?_DELAY1MS?MAIN

?PR?DRIVE?MAIN
  +--> ?PR?_DELAY?MAIN

?PR?CLOSE?MAIN
  +--> ?PR?_DELAY1MS?MAIN



SYMBOL TABLE OF MODULE:  Table_lamps (MAIN)

  VALUE           TYPE          NAME
  ----------------------------------

  -------         MODULE        MAIN
  C:0000H         SYMBOL        _ICE_DUMMY_
  D:0090H         PUBLIC        P1
  D:00A0H         PUBLIC        P2
  B:00D0H.6       PUBLIC        AC
  B:00B0H.4       PUBLIC        T0
  B:00B0H.5       PUBLIC        T1
  B:00A8H.7       PUBLIC        EA
  B:0090H.0       PUBLIC        T2
  B:0080H.0       PUBLIC        P0_0
  B:0090H.0       PUBLIC        P1_0
  B:0080H.1       PUBLIC        P0_1
  B:00D0H.1       PUBLIC        FL
  B:00A0H.0       PUBLIC        P2_0
  B:0090H.1       PUBLIC        P1_1
  B:0080H.2       PUBLIC        P0_2
  B:00B0H.0       PUBLIC        P3_0
  B:00A0H.1       PUBLIC        P2_1
  B:0090H.2       PUBLIC        P1_2
  B:0080H.3       PUBLIC        P0_3
  B:00B0H.1       PUBLIC        P3_1
  B:00A0H.2       PUBLIC        P2_2
  B:0090H.3       PUBLIC        P1_3
  B:0080H.4       PUBLIC        P0_4
  B:00B0H.2       PUBLIC        P3_2
  B:00A0H.3       PUBLIC        P2_3
  B:0090H.4       PUBLIC        P1_4
  B:0080H.5       PUBLIC        P0_5
  B:00C8H.6       PUBLIC        EXF2
  B:00B0H.7       PUBLIC        RD
  B:00B0H.3       PUBLIC        P3_3
  B:00A0H.4       PUBLIC        P2_4
  B:0090H.5       PUBLIC        P1_5
  B:0080H.6       PUBLIC        P0_6
  B:00B0H.4       PUBLIC        P3_4
  B:00A0H.5       PUBLIC        P2_5
  B:0090H.6       PUBLIC        P1_6
  B:0080H.7       PUBLIC        P0_7
  B:00B0H.5       PUBLIC        P3_5
  B:00A8H.4       PUBLIC        ES
  B:00A0H.6       PUBLIC        P2_6
BL51 BANKED LINKER/LOCATER V4.13                                                      12/03/2007  00:32:50  PAGE 3


  B:0090H.7       PUBLIC        P1_7
  C:0094H         PUBLIC        close
  B:00B0H.6       PUBLIC        P3_6
  B:00A0H.7       PUBLIC        P2_7
  B:00B0H.7       PUBLIC        P3_7
  B:0098H.0       PUBLIC        RI
  B:00D0H.7       PUBLIC        CY
  B:00B0H.2       PUBLIC        INT0
  C:0055H         PUBLIC        drive
  B:00B0H.3       PUBLIC        INT1
  B:0098H.1       PUBLIC        TI
  D:0008H         PUBLIC        Brightness
  B:00B8H.4       PUBLIC        PS
  B:0090H.1       PUBLIC        T2EX
  B:00D0H.2       PUBLIC        OV
  C:003BH         PUBLIC        main
  B:00C8H.1       PUBLIC        C_T2
  B:00B0H.6       PUBLIC        WR
  C:0020H         PUBLIC        add
  B:0020H.0       PUBLIC        MARK
  C:0003H         PUBLIC        dec
  B:00C8H.5       PUBLIC        RCLK
  B:00C8H.4       PUBLIC        TCLK
  C:0081H         PUBLIC        open
  C:00A7H         PUBLIC        init
  B:0088H.1       PUBLIC        IE0
  B:0088H.3       PUBLIC        IE1
  C:006CH         PUBLIC        _Delay1mS
  B:00C8H.0       PUBLIC        CP_RL2
  B:00A0H.1       PUBLIC        ADD
  B:00A8H.1       PUBLIC        ET0
  B:00A8H.3       PUBLIC        ET1
  B:0088H.5       PUBLIC        TF0
  B:00A8H.5       PUBLIC        ET2
  B:0088H.7       PUBLIC        TF1
  B:00A0H.2       PUBLIC        DEC
  B:00C8H.7       PUBLIC        TF2
  B:0098H.2       PUBLIC        RB8
  B:00A8H.0       PUBLIC        EX0
  B:0088H.0       PUBLIC        IT0
  B:00A8H.2       PUBLIC        EX1
  B:0098H.3       PUBLIC        TB8
  B:0088H.2       PUBLIC        IT1
  B:00D0H.0       PUBLIC        P
  B:0098H.7       PUBLIC        SM0
  B:0098H.6       PUBLIC        SM1
  B:0098H.5       PUBLIC        SM2
  B:00B8H.1       PUBLIC        PT0
  B:0090H.0       PUBLIC        LED
  B:00D0H.3       PUBLIC        RS0
  B:00B8H.3       PUBLIC        PT1
  B:00D0H.4       PUBLIC        RS1
  B:00B8H.5       PUBLIC        PT2
  B:0088H.4       PUBLIC        TR0
  B:0088H.6       PUBLIC        TR1
  B:00C8H.2       PUBLIC        TR2
  B:00B8H.0       PUBLIC        PX0
BL51 BANKED LINKER/LOCATER V4.13                                                      12/03/2007  00:32:50  PAGE 4


  B:00B8H.2       PUBLIC        PX1
  B:00C8H.3       PUBLIC        EXEN2
  B:0098H.4       PUBLIC        REN
  B:00B0H.0       PUBLIC        RXD
  B:00B0H.1       PUBLIC        TXD
  C:00B8H         PUBLIC        _delay
  B:00D0H.5       PUBLIC        F0
  B:00A0H.0       PUBLIC        ONOFF
  -------         PROC          _DELAY1MS
  D:0006H         SYMBOL        a
  -------         DO            a
  D:0005H         SYMBOL        i
  -------         ENDDO         i
  C:006CH         LINE#         24
  C:006CH         LINE#         26
  C:0075H         LINE#         27
  C:0080H         LINE#         28
  C:0080H         LINE#         29
  -------         ENDPROC       _DELAY1MS
  -------         PROC          _DELAY
  D:0007H         SYMBOL        d
  -------         DO            d
  D:0006H         SYMBOL        i
  -------         ENDDO         i
  C:00B8H         LINE#         33
  C:00B8H         LINE#         35
  C:00BCH         LINE#         36
  C:00C7H         LINE#         37
  C:00C7H         LINE#         38
  -------         ENDPROC       _DELAY
  -------         PROC          DRIVE
  -------         DO            DRIVE
  D:0005H         SYMBOL        a
  -------         ENDDO         a
  C:0055H         LINE#         42
  C:0055H         LINE#         44
  C:0057H         LINE#         45
  C:0059H         LINE#         46
  C:005EH         LINE#         47
  C:0061H         LINE#         48
  C:0063H         LINE#         49
  C:0068H         LINE#         50
  C:006BH         LINE#         51
  -------         ENDPROC       DRIVE
  -------         PROC          OPEN
  C:0081H         LINE#         55
  C:0081H         LINE#         56
  C:0084H         LINE#         57
  C:008BH         LINE#         58
  C:008EH         LINE#         59
  C:0090H         LINE#         60
  C:0093H         LINE#         61
  C:0093H         LINE#         62
  C:0093H         LINE#         63
  -------         ENDPROC       OPEN
  -------         PROC          CLOSE
  C:0094H         LINE#         67
BL51 BANKED LINKER/LOCATER V4.13                                                      12/03/2007  00:32:50  PAGE 5


  C:0094H         LINE#         68
  C:0097H         LINE#         69
  C:009EH         LINE#         70
  C:00A1H         LINE#         71
  C:00A3H         LINE#         72
  C:00A6H         LINE#         73
  C:00A6H         LINE#         74
  C:00A6H         LINE#         75
  -------         ENDPROC       CLOSE
  -------         PROC          ADD
  C:0020H         LINE#         79
  C:0020H         LINE#         80
  C:0023H         LINE#         81
  C:002BH         LINE#         82
  C:0034H         LINE#         83
  C:003AH         LINE#         84
  C:003AH         LINE#         85
  C:003AH         LINE#         86
  -------         ENDPROC       ADD
  -------         PROC          DEC
  C:0003H         LINE#         90
  C:0003H         LINE#         91
  C:0006H         LINE#         92
  C:000EH         LINE#         93
  C:0019H         LINE#         94
  C:001FH         LINE#         95
  C:001FH         LINE#         96
  C:001FH         LINE#         97
  -------         ENDPROC       DEC
  -------         PROC          INIT
  C:00A7H         LINE#         101
  C:00A7H         LINE#         102
  C:00A9H         LINE#         103
  C:00ABH         LINE#         104
  C:00ADH         LINE#         105
  C:00AFH         LINE#         106
  C:00B5H         LINE#         107
  C:00B7H         LINE#         108
  -------         ENDPROC       INIT
  -------         PROC          MAIN
  C:003BH         LINE#         112
  C:003BH         LINE#         113
  C:003EH         LINE#         114
  C:003EH         LINE#         115
  C:0041H         LINE#         116
  C:0044H         LINE#         117
  C:0044H         LINE#         118
  C:0047H         LINE#         119
  C:004AH         LINE#         120
  C:004DH         LINE#         121
  C:0050H         LINE#         122
  C:0053H         LINE#         123
  C:0053H         LINE#         124
  -------         ENDPROC       MAIN
  -------         ENDMOD        MAIN

LINK/LOCATE RUN COMPLETE.  0 WARNING(S),  0 ERROR(S)
